:100000000C94F6000C9415010C9415010C94150138
:100010000C9415010C94E4030C9415010C94150137
:100020000C9415010C9415010C9415010C941501F8
:100030000C94031A0C9415010C9415010C941501E1
:100040000C94BD030C9415010C9417010C9415012C
:100050000C9415010C9415010C9415010C941501C8
:100060000C9415010C9415010C9415010C941501B8
:100070000C9415010C9415010C9415010C941501A8
:100080000C9415010C9415010C941501001002102C
:100090000410061008100A100C100E101010121088
:1000A0001410161018101A101C101E1020102210F8
:1000B0002410661066106610661066106610261012
:1000C00028102A102C102E10301032103410381036
:1000D0003C10421046104A104E10521058105A1040
:1000E0005C106010AF10B110B310B510B710B9109C
:1000F000BB10BD10BF10C110C310C510C710C91070
:10010000CB10CD10CF10D110D31015111511151122
:10011000151115111511D510D710D910DB10DD10E0
:10012000DF10E110E310E710EB10F110F510F910FB
:10013000FD100111071109110B110F118111871108
:100140008D11931199119F11A511AB11B111B71117
:10015000BD11C311C911CF11D511DB11E111E71187
:10016000ED117E117E117E117E117E117E11F31133
:10017000F911FF1105120B12111217121D1227127D
:1001800033123D12471251125B1265126F12751233
:100190007B128112CA12CD12D012D312D612D912EA
:1001A000DC12DF12E212E512E812EB12EE12F1128B
:1001B000F412F712FA12FD120013C712C712C71277
:1001C000C712C712C7120313061309130C130F1318
:1001D000181315131213151318131B131E132113C1
:1001E00027132413241327132A132D1311241FBE9E
:1001F000CFEFD0E1DEBFCDBF13E0A0E0B1E0E6E598
:10020000FAE300E00BBF02C007900D92AC33B107D8
:10021000D9F716E0ACE3B3E001C01D92A237B107F5
:10022000E1F70E942C010C942A1D0C9400001F92EF
:100230000F920FB60F9211240F900FBE0F901F90C8
:100240001895FC0120E030E002C02F5F3F4F819104
:100250008823D9F7C9010895CCEFD0E1DEBFCDBF27
:10026000F8940E9453090E94CC0E8FEF87BB88BB85
:10027000C7980E94B80981E897E10E94030A85E6C1
:100280009CE00E94080A81E090E00E940D0ADE01D5
:100290001196E6EFF2E083E001900D928150E1F7D4
:1002A000CE0101960E94020E80E091E00E949E0E17
:1002B00081E191E00E94960E82E491E00E948E0E10
:1002C0000E94D80D4C0164E670E00E941B0A60E0B9
:1002D00070E0C4010E94440D3C0140E050E0BC01CC
:1002E000C4010E943C0A2EE0A22E22E0B22ECC24B1
:1002F000DD2490E4E92EF12C02E021E030E041E041
:1003000050E0B301C4010E94D90C8DE2A82E83E015
:10031000B82E21E030E041E050E0B301C4010E947A
:10032000110D10929A031092990310929C0310924F
:100330009B030E940E1B8FE784BB8AE285BB0E9451
:10034000080485E585BB0E94080415BA0E94520F77
:100350000E9453090E94D10E7894FFCF0F931F93F0
:10036000CF93DF93EC018134910510F18091A503C7
:100370009091A603892BE1F4DF93CF938BE491E076
:100380009F938F930E94071B1092A2031092A103C8
:10039000D093A403C093A30381E090E09093A603BD
:1003A0008093A503C0E4D0E00F900F900F900F90C2
:1003B00068E08BE20E94A10900E010E00EC0E0912D
:1003C000A103F091A203E00FF11FE551FB4F608103
:1003D00089E20E94A1090F5F1F4F0C171D0779F7D3
:1003E0008091990390919A03019749F467E08BE219
:1003F0000E94A10910929A03109299030AC063E027
:100400008BE20E94A10981E090E090939A0380938F
:100410009903DF91CF911F910F910895CF93DF93AF
:100420008091A5039091A603019709F04CC088E73D
:1004300091E09F938F930E94071B2091A10330911D
:10044000A2038091A3039091A4030F900F9028170B
:100450003907C8F586E991E09F938F930E94071BA7
:10046000C091A303D091A4038091A1039091A20312
:10047000C81BD90B8091A1039091A203805C9F4F70
:100480009093A2038093A1030F900F90C134D105E4
:100490005CF08FEB91E09F938F930E94071B80E4A9
:1004A00090E00E94AE010DC08BED91E09F938F9381
:1004B0000E94071BCE010E94AE011092A60310926B
:1004C000A5030F900F90DF91CF9108950F931F9385
:1004D000CF93DF938C011092A2031092A10310928C
:1004E000A6031092A503C79AFC018081282F2295AC
:1004F0002F70C22FDD2799279F938F93DF93CF9380
:1005000088EE91E09F938F930E94071B8DB79EB753
:1005100006960FB6F8949EBF0FBE8DBFC430D105AE
:1005200009F451C0C530D10584F4C130D10569F159
:10053000C230D1051CF4CD2BC1F074C0C230D1053E
:1005400071F1239709F06EC034C0C630D10509F4AB
:100550004EC0C630D1050CF440C0C730D10509F4F7
:1005600050C0289709F05EC053C0F80180818630E2
:1005700041F48281813009F06AC0C8010E94D0191B
:1005800066C0C8010E944B0F62C088E092E09F9352
:100590008F930E94071BC8010E940F1456C08BE165
:1005A00092E09F938F930E94071BC8010E945315EE
:1005B0004CC08FE292E09F938F930E94071BC8016B
:1005C0000E94731642C083E492E09F938F930E942F
:1005D000071BC8010E94EE1738C087E592E09F9381
:1005E0008F930E94071BC8010E94D51A2EC08BE171
:1005F00092E09F938F930E94071BC8010E94E5051C
:1006000024C08BE692E09F938F930E94071B1DC02E
:1006100083E992E09F938F930E94071BC8010E9479
:10062000B91B13C08AEA92E09F938F930E94071B25
:10063000F80180818093EB0483E08093EC041092B6
:10064000ED0483E090E00E94AE010F900F90C798F8
:10065000DF91CF911F910F9108950F931F93CF9327
:10066000DF93EC018C010F5F1F4F898199279F93C6
:100670008F9387EB92E09F938F930E94071B80914B
:100680009B0390919C030F900F900F900F900197F8
:1006900091F58BED92E09F938F930E94071B20E0D2
:1006A00030E00F900F90E0919D03F0919E03E20FD8
:1006B000F31FDE01A20FB31F8C91E555FC4F808321
:1006C0002F5F3F4F2034310571F780919D0390914A
:1006D0009E03805C9F4F90939E0380939D03209187
:1006E0009D0330919E0380919F039091A003281752
:1006F0003907F0F128C085EE92E09F938F930E9416
:10070000071B10929E0310929D0320E030E00F9093
:100710000F90E0919D03F0919E03E20FF31FDE0125
:10072000A20FB31F8C91E555FC4F80832F5F3F4F85
:100730002034310571F730939E0320939D03F80117
:100740002081203448F410929C0310929B038BEA82
:1007500093E00E9466020CC081E090E090939C03BD
:1007600080939B03822F99279093A00380939F03EC
:10077000DF91CF911F910F9108951F920F920FB6A5
:100780000F9211242F933F934F935F936F937F9317
:100790008F939F93AF93BF93EF93FF930E941C0F90
:1007A0008091450382BFFF91EF91BF91AF919F91DF
:1007B0008F917F916F915F914F913F912F910F900A
:1007C0000FBE0F901F9018951F920F920FB60F92A9
:1007D00011242F933F934F935F936F937F938F9346
:1007E0009F93AF93BF93EF93FF930E94A60EFF9149
:1007F000EF91BF91AF919F918F917F916F915F9199
:100800004F913F912F910F900FBE0F901F90189511
:1008100020E080E49CE90197F1F72F5F2931C9F7C7
:100820000895882329F0813069F084E090E00895EC
:100830008EE080936F038093700388E18AB981E032
:1008400090E008958EE0809354038093550388E1EF
:1008500080939A0081E090E00895882329F0813008
:1008600081F084E090E0089510926F03109270037D
:100870001092900019B81AB81092950081E090E09B
:1008800008951092540310925503109298001092FC
:10089000990010929A0010929D0081E090E00895D6
:1008A0000F93882329F0813039F084E090E00AC06A
:1008B0002093900069B904C0209398006093990038
:1008C00081E090E00F910895623011F492E001C050
:1008D00090E0882329F0813071F084E090E0089561
:1008E00080919500990F990F990F982B90939500EF
:1008F00081E090E0089580919D00990F990F990FE4
:10090000982B90939D0081E090E00895663061F00F
:10091000673019F0653019F404C021E003C021E00C
:1009200004C020E090E002C020E091E0882329F09C
:10093000813079F084E090E0089580919500220F55
:10094000220F990F922B982B9093950081E090E0C5
:10095000089580919D00220F220F990F922B982BC2
:1009600090939D0081E090E00895653439F06F34F4
:1009700019F421E091E004C020E001C021E090E002
:10098000882329F0813089F084E090E008958091F7
:1009900095002295220F207E9295907F922B982B86
:1009A0009093950081E090E0089580919D002295BC
:1009B000220F207E9295907F922B982B90939D00F2
:1009C00081E090E00895882329F0813049F084E0A7
:1009D00090E008955D9BFECF6CB981E090E00895B2
:1009E00080919B0085FFFCCF60939C0081E090E0AC
:1009F0000895FF920F931F93CF93DF93F82EEB018F
:100A00008A0181E08F1548F484E090E00DC0F80180
:100A100061918F018F2D0E94E3042197FFEFCF3F5B
:100A2000DF07A9F781E090E0DF91CF911F910F914F
:100A3000FF900895882329F0813039F084E090E018
:100A400008955F9BFECF8CB106C080919B0087FF0D
:100A5000FCCF80919C0099270895FF920F931F93DC
:100A6000CF93DF93F82E8B0181E08F1518F484E08B
:100A700090E00EC0EA0107C08F2D0E941A05F80110
:100A800081938F0121971C161D06B4F381E090E03D
:100A9000DF91CF911F910F91FF90089577270E94CA
:100AA000F9048093EC041092ED0483E090E00E943E
:100AB000AE0108950E9486048093EC041092ED0428
:100AC00083E090E00E94AE0108950E948604809326
:100AD000EC041092ED0483E090E00E94AE010895D2
:100AE0000E9464048093EC041092ED0483E090E093
:100AF0000E94AE0108950F930E9450048093EC046D
:100B00001092ED0483E090E00E94AE010F910895F1
:100B10000E942D048093EC041092ED0483E090E099
:100B20000E94AE0108950E9411048093EC0410927B
:100B3000ED0483E090E00E94AE010895CF92DF9231
:100B4000EF92FF920F931F93CF93DF93CDB7DEB752
:100B50008B01CDB6DEB62DB73EB7261B370B0FB6D1
:100B6000F8943EBF0FBE2DBFEDB6FEB60894E11C53
:100B7000F11CAB01B7010E942D058093EC0420E02D
:100B800030E00AC0F701E20FF31F8081F901E35161
:100B9000FB4F80832F5F3F4F201731079CF3F801F5
:100BA000E351FB4F1082C80103960E94AE010FB6BD
:100BB000F894DEBE0FBECDBEDF91CF911F910F9195
:100BC000FF90EF90DF90CF9008950F93FC0180810C
:100BD0008093EB04843611F1853648F48236B1F007
:100BE0008336E0F4803651F0813681F50BC08736CC
:100BF00039F18836E9F0853649F515C082810E94C1
:100C000093052DC082810E94880529C00681258117
:100C10004481638182810E947B0521C0638182813E
:100C20000E9470051CC0638182810E945A0517C012
:100C3000AF014C5F5F4F638182810E944E050FC000
:100C40006381772782810E949E0509C083E080939B
:100C5000EC041092ED0483E090E00E94AE010F914D
:100C6000089587E28093530685E28093520690E2CE
:100C7000909354061092550628E030E030935706C2
:100C80002093560683E280935F0681E280935E069E
:100C9000909360061092610630936306209362067B
:100CA0000895089560916B0681E20E94A10908955C
:100CB00068E08BE20E94A10961E188E20E94A1093B
:100CC00068E08FE20E94A10961E18CE20E94A10923
:100CD00061E08FE20E94A10910929A031092990399
:100CE00065E083E20E94A10908950F931F938C0190
:100CF00060E480E20E94A109F8016281605884E00A
:100D00000E94A109F801828180936A061F910F91C8
:100D100008950F931F93CF93DF93EC0128853985B6
:100D200012161306DCF58E819F81821793071CF53E
:100D300068E083E20E94A10900E010E00FC08A850C
:100D40009B85E80FF91F608181E20E94A1098E81D5
:100D50009F8101969F838E830F5F1F4FEE81FF81DE
:100D600088859985083011051CF4E817F9073CF3CC
:100D7000E817F90724F061E087E20E94A1098B815E
:100D8000813031F465E089810E94A1091B8206C08F
:100D900061E089810E94A10981E08B83DF91CF917D
:100DA0001F910F910895CF93DF93CDB7DEB72497AE
:100DB0000FB6F894DEBF0FBECDBFDC01FC0122816F
:100DC0003381109265061092640681E0809361067B
:100DD000832F99278230D9F0833069F1813009F06F
:100DE00057C080913E0699279093670680936606C8
:100DF0008EE396E0909369068093680686819781DA
:100E00008034910509F044C088E090E029C0FD01DC
:100E1000868197819093670680936606E22FFF276D
:100E2000EE0FFF1F8091500690915106E80FF91FB9
:100E30008081918129C02223C1F0E22FFF27EE0F8C
:100E4000FF1F8091A9039091AA03E80FF91F019059
:100E5000F081E02DF0936906E09368068081992780
:100E6000909367068093660613C094E0998383E0AD
:100E70008A8389E08B839C8384E090E0909367066B
:100E800080936606CE01019690936906809368066A
:100E90008EE596E00E94890624960FB6F894DEBF90
:100EA0000FBECDBFDF91CF910895CF93DF9382E244
:100EB0000E947809C82FDD27C5FF1AC068E083E2C9
:100EC0000E94A109C6FF10C02091640630916506FA
:100ED0008091660690916706281739072CF48EE5F5
:100EE00096E00E94890604C061E087E20E94A109A1
:100EF000DF91CF9108951F93CF93DF9388E00E94F5
:100F00007809182FC82FDD27C6FF18C060E085E0DC
:100F10000E94A10960E884E00E94A10960E080E2EB
:100F20000E94A10968E083E20E94A10961E087E2D2
:100F30000E94A10962E085E00E94A109C4FF04C0EB
:100F400060EC89E00E94A10917FF04C060ED89E010
:100F50000E94A109DF91CF911F9108958AE00E941C
:100F60007809992780FF03C00E945507089581FFE3
:100F70000DC08AE20E94780980912B06813061F4CD
:100F8000E0912E06F0912F060995089582E30E94C4
:100F900078098AE30E94780908958EE00E94780912
:100FA00068E08FE20E94A10961E08FE20E94A1093E
:100FB00020916606309167068091620690916306E3
:100FC000821793075CF468E083E20E94A10961E064
:100FD00087E20E94A10981E0809361060895AF92A3
:100FE000BF92CF92DF92EF92FF920F931F93CF9316
:100FF000DF93CDB7DEB728970FB6F894DEBF0FBEEC
:10100000CDBF86E20E94780986FF7EC08E010F5F09
:101010001F4F580169E0C62ED12CCC0EDD1E8091E9
:1010200052060E947809F80181938F017501EC1531
:10103000FD05A9F768E087E20E94A10968E083E264
:101040000E94A10980E20E9478098F77682F80E2D0
:101050000E94A1098981992780769070803291053C
:1010600009F440C080349105D1F1892BF1F5F501E7
:1010700081818630D9F0873048F48130F1F18130B8
:10108000C8F08330D1F1853081F521C0893019F164
:101090008A3018F4883049F505C08A3071F18B30F8
:1010A00021F520C0C5010E94520627C0C5010E943B
:1010B000D30623C068E083E20E94A10961E081E2D7
:1010C0000E94A10960E081E20E94A1090BC0C50154
:1010D0000E94750612C0C5010E9458060EC0C501C7
:1010E0000E94510965E083E206C080E20E9478090F
:1010F0008058682F80E20E94A109F701808188232F
:10110000D1F465E083E215C0209166063091670650
:1011100080916206909163068217930764F410929F
:1011200067061092660668E083E20E94A10961E00A
:1011300087E20E94A10928960FB6F894DEBF0FBE81
:10114000CDBFDF91CF911F910F91FF90EF90DF9076
:10115000CF90BF90AF900895CF92DF92EF92FF9221
:101160000F931F93CF93DF93CDB7DEB7C054D0401A
:101170000FB6F894DEBF0FBECDBF8CE00E94780999
:10118000992780FF03C00E94EF077BC081FF2AC020
:101190008EE20E9478098DE20E94780989838E018F
:1011A0000F5F1F4F6801FFE3EF2EF12CE00EF11EE1
:1011B0000F5F1F4F0E946409F80180830E151F0501
:1011C000B9F780913C03813031F4E0913F03F09115
:1011D0004003C601099568E08FE20E94A10961E021
:1011E0008FE22BC082FF2CC086E30E94780985E342
:1011F0000E94780989838E010F5F1F4F6801EFE31A
:10120000EE2EF12CE00EF11E0F5F1F4F0E946409BD
:10121000F80180830E151F05B9F780913D038130D9
:1012200031F4E0914103F0914203C601099568E071
:1012300087E30E94A10961E087E30E94A10921C020
:1012400083FF1FC08EE30E9478098E010F5F1F4F3E
:10125000680171E4E72EF12CEC0EFD1E8DE30E9477
:101260007809F80181938F01EE15FF05B9F7809198
:101270003E03813031F4E0913F03F0914003C60119
:101280000995C05CDF4F0FB6F894DEBF0FBECDBF2F
:10129000DF91CF911F910F91FF90EF90DF90CF9052
:1012A00008950895089581E08ABF80E189BFE4E64A
:1012B000F0E0808187608083E5E6F0E080818360F4
:1012C0008083A79AAF9A089585B3805885BBE5E6D9
:1012D000F0E0808122E0822780830000000089B353
:1012E00095B3905895BB9081922790839927089544
:1012F0009FEF9ABB8BBB85B3805885BBE5E6F0E0DA
:10130000808195E08927808385B3805885BB808163
:101310008927808300001ABA0E94640999270895DA
:101320008BBB85B3805885BBE5E6F0E0808191E01A
:101330008927808385B3805885BB808189278083F6
:1013400008958BBB8FEF8ABB85B3805885BBE5E6DC
:10135000F0E0808195E08927808385B3805885BB44
:10136000808189278083862F0E949009089508959F
:1013700082E180933E0681E080933F0680E191E028
:1013800090934106809340061092420610924306C5
:101390001092440688E0809345061092470610920A
:1013A0004606109249061092480610924B0610927B
:1013B0004A0610924C0610924D0610924E0610925C
:1013C0004F0610923C0310923D0310923E03109280
:1013D0002B0610922C0610922D06109235061092B4
:1013E00034061092A8031092A7030895909347061D
:1013F00080934606709349066093480650934B06C7
:1014000040934A06089590934706809346060895B0
:101410009093490680934806089590934B068093D5
:101420004A060895809342060895809343060895DE
:10143000809344060895CF93DF939C01CB01E09104
:101440003406F091350662E070E00E94031D0FC083
:10145000A081B1818281823039F4ED018D8199279B
:101460008217930709F468870780F085E02D30978D
:1014700079F7DF91CF910895CF93DF939C01E091AD
:101480003406F091350614C0A081B1818281843088
:1014900061F4848199278217930739F4868199270B
:1014A0008617970711F4ED014B830780F085E02D37
:1014B000309751F7DF91CF910895BF92CF92DF928D
:1014C000EF92FF920F931F93CF93DF936C01162F30
:1014D000F42EB22EC0913406D09135062097A1F497
:1014E00089E090E00E94051CFC01909335068093F2
:1014F0003406D182C082138310861782F282B482AE
:101500000583E68215C0EC018F8198850097D9F795
:1015100089E090E00E94051CFC0198878F83D182AE
:10152000C0821383F282B4820583E682108617821A
:10153000DF91CF911F910F91FF90EF90DF90CF90AF
:10154000BF900895EF92FF921F93CF93DF937C019A
:10155000C091A703D091A803209711F011E012C009
:1015600085E090E00E94051CFC019093A803809305
:10157000A703F182E08212821482138210E012C06B
:101580001F5FEC018B819C810097D1F785E090E093
:101590000E94051CFC019C838B83F182E0821283F4
:1015A00014821382812F9927DF91CF911F91FF9091
:1015B000EF900895EF92FF920F931F93CF93DF93D5
:1015C000E091A703F091A80380E090E00380F4810C
:1015D000E02D01963097D1F7880F991F0E94051CC6
:1015E0009093AA038093A9030091A7031091A803E5
:1015F000E801E880F9808A81C82FDD27CC0FDD1F44
:101600008091A9039091AA03C80FD91FF701808187
:1016100099270E94051C9983888320E030E017C039
:10162000E801EA81FF27EE0FFF1F8091A903909147
:10163000AA03E80FF91F0190F081E02DE20FF31FDC
:10164000D701A20FB31F8C9180832F5F3F4FF7010B
:1016500080819927281739071CF3E8018B819C8129
:10166000009711F08C01C4CFDF91CF911F910F91A2
:10167000FF90EF9008954F925F926F927F928F92BA
:101680009F92AF92BF92CF92DF92EF92FF920F9311
:101690001F93CF93DF93E0913406F09135066624D3
:1016A000772409C08281823019F40894611C711C6E
:1016B0000780F085E02D3097A9F74301880C991C2D
:1016C000C4010E94051C9093510680935006E1E0EE
:1016D000EE2EF12CAA24BB2455C0E0913406F091E3
:1016E000350679E0C72ED12C15C0A081B181848147
:1016F00099278E159F0519F48381C80ED11CED0121
:101700008D818E1521F48281823009F45D0107807C
:10171000F085E02D309749F7009150061091510661
:1017200002501040080D191DC6010E94051CF80149
:101730009183808320E030E0E0915006F0915106E3
:10174000E80DF91D32970190F081E02DE20FF31FB3
:10175000D501A20FB31F8C9180832F5F3F4F29309B
:10176000310551F7E0915006F0915106E80DF91D51
:1017700032970190F081E02D8C2D875F8283089451
:10178000E11CF11C6E147F040CF0A7CF61E0C62EA3
:10179000D12C59E0A52EB12C4424552442E0842EAE
:1017A000912CA1C0A0913406B091350612C0ED91E4
:1017B000FC9111978181823049F4858199278C159C
:1017C0009D0521F48481482E552405C0ED01AF818B
:1017D000B885109761F731E0E32EF12C79C0609164
:1017E0003406709135066DC0FB01C081D1818981BD
:1017F000843009F063C0868199278E159F0509F012
:101800005DC0848199278C159D0509F057C095010D
:1018100040E050E0E0915006F0915106E80DF91DCE
:1018200032970190F081E02DE20FF31FDE01A40F4B
:10183000B51F8C9180832F5F3F4F4F5F5F4F4930C3
:10184000510541F789E090E0A80EB91EC091340619
:10185000D091350631C08A81853059F58C81992720
:101860008C159D0531F58D8199278E159F0509F5FC
:1018700008811981950140E050E0E0915006F09117
:101880005106E80DF91D32970190F081E02DE20F2D
:10189000F31FD801A40FB51F8C9180832F5F3F4F9A
:1018A0004F5F5F4F4730510541F7E7E0F0E0AE0E84
:1018B000BF1E0F80D885C02D209769F6EB016F8180
:1018C00078856115710509F08FCF0894E11CF11C32
:1018D0004E145F040CF083CF0894C11CD11CE2E0CD
:1018E000F0E08E0E9F1E6C147D040CF05BCFDF9138
:1018F000CF911F910F91FF90EF90DF90CF90BF900D
:10190000AF909F908F907F906F905F904F900895D1
:101910006F927F928F929F92AF92BF92CF92DF92FF
:10192000EF92FF920F93CF93DF935C013B0149014C
:10193000E0913406F091350616C0A081B181848112
:101940009927A816B90661F4868199278615970507
:1019500039F48281843021F4ED018C818F5F8C8396
:101960000780F085E02D309741F787E090E00E94F6
:10197000051CFC0187E0808385E0818382820383EC
:10198000F582E482C682EE24062D2A2D45E067E02A
:10199000CF010E945D0ADF91CF910F91FF90EF90F0
:1019A000DF90CF90BF90AF909F908F907F906F907F
:1019B0000895AF92BF92CF92DF92EF92FF920F9372
:1019C000FC01A114B10401F14230510571F0433022
:1019D000510599F041305105B9F481E080932B060F
:1019E000B0922F06A0922E060FC081E080932C06A5
:1019F000B0923106A092300607C081E080932D0698
:101A0000B0923306A092320620583F4FCF010E9479
:101A1000880C0F91FF90EF90DF90CF90BF90AF9028
:101A20000895AF92BF92CF92DF92EF92FF920F9301
:101A3000FC014230510571F04330510599F04130BD
:101A40005105B9F481E080933C03B0924003A09229
:101A50003F030FC081E080933D03B0924203A09208
:101A6000410307C081E080933E03B0924403A092FB
:101A70004303CF010E94880C0F91FF90EF90DF90FD
:101A8000CF90BF90AF900895CF92DF92EF920F93D7
:101A90001F93CF93DF936C018B01A0913406B0911B
:101AA0003506C0E0D0E014C02D913C911197F901AA
:101AB00085818C1551F4FD018281823031F4F90168
:101AC00084818F5F8483C82FDD27FD01A781B085C6
:101AD000109751F789E090E00E94051CFC0189E015
:101AE000808384E0818302831382148215821682AC
:101AF00017821086EC2E00E02C2D44E069E0CF0127
:101B00000E945D0ACE01DF91CF911F910F91EF905E
:101B1000DF90CF900895BF92CF92DF92EF92FF9225
:101B20000F931F93CF93DF936C017B01142FB22E81
:101B3000A0913406B0913506C0E0D0E014C02D91DC
:101B40003C911197F90185818C1551F4FD01828139
:101B5000823031F4F90184818F5F8483C82FDD27BF
:101B6000FD01A781B085109751F789E090E00E94B0
:101B7000051CFC0189E0808384E08183E28213827A
:101B800014821583B68207831086EC2E00E02C2D7C
:101B900044E069E0CF010E945D0ACE01DF91CF9160
:101BA0001F910F91FF90EF90DF90CF90BF9008951D
:101BB000EF920F931F9310914F061F5F10934F06E4
:101BC00089E090E00E94051CFC0189E0808389E0A7
:101BD00090E09383828382E081831482158316824E
:101BE00080EA87838AE18087EE2400E020E042E0FB
:101BF00069E0CF010E945D0A812F99271F910F9103
:101C0000EF900895CF93DF93EC01FC010190002049
:101C1000E9F7E81BF90BCF01880F991F0E94051CFB
:101C20009C01FE0101900020E9F7EC1BFD0BEE0F7B
:101C3000FF1FDC01EC9383E0F901818340E050E079
:101C400009C0FE01E40FF51F80818C93FD01118214
:101C50004F5F5F4F1296FE0101900020E9F7319728
:101C6000EC1BFD0B4E175F0760F3C9010E94A20A2F
:101C70009927DF91CF910895EF92FF920F931F93D1
:101C8000CF93DF938C017B01CA010E94020E9C015D
:101C9000E0913406F091350614C0A081B1818281B3
:101CA000843061F4848199278017910739F4868103
:101CB00099278E159F0511F4ED0128870780F0857F
:101CC000E02D309751F7DF91CF911F910F91FF9049
:101CD000EF9008950F931F93CF93DF938C01CB0167
:101CE0000E94020E9C01E0913406F09135060FC06F
:101CF000A081B1818281823039F4ED018D819927F3
:101D00008017910709F42E830780F085E02D309726
:101D100079F7DF91CF911F910F9108950E94020EE4
:101D20001816190614F480934E0608950E94020EA8
:101D30001816190614F480934D0608950E94020E99
:101D40001816190614F480934C0608951F9386E024
:101D50000E947809992786FF03C00E94AC080EC034
:101D600082FF03C00E94AE0709C081FF03C00E942A
:101D70007B0704C084FF02C00E94CD0787E00E9459
:101D80007809182F60E087E00E94A109612F87E0A1
:101D90000E94A1091F91089562E081E00E94A109BB
:101DA00008950E943B0B0E94DA0A0E94310661E00E
:101DB00080E00E94A10980E00E94780980FDFBCFAD
:101DC00062E081E00E94A10960E884E00E94A1092C
:101DD00060E480E20E94A10968E083E20E94A10918
:101DE00069E087E20E94A1096FE08DE00E94A109ED
:101DF0006FE08BE00E94A10968ED89E00E94A109D3
:101E000063E38FE00E94A10966ED87E00E94A109CB
:101E100062E085E00E94A1096CEC80E00E94A109CB
:101E200008958EEC8093450381E087BF8091450340
:101E300082BF83E083BF08950895089583E080936F
:101E4000EB0481E08093EC048BE08093ED049FE64B
:101E50009093EE0483E68093EF0484E78093F0048C
:101E60009093F10480E78093F20485E78093F30474
:101E700083E78093F4048FE58093F50480E38093F7
:101E8000F60481E38093F7041092F8048EE090E06A
:101E90000E94AE010895FC018081833011F40E94FC
:101EA0001E0F08951F9311E0812F0E94751060E0AE
:101EB000812F0E9462111F5F1431B1F718E1812F49
:101EC0000E94751060E0812F0E9462111F5F1B321B
:101ED000B1F71F910895CF93DF93DC01EC01EA8104
:101EE000FB8121918E81815019F48981E81BF109D0
:101EF000ED01FB83EA838E839FB7F8948C91815028
:101F00008C939FBF822F9927DF91CF910895FC0179
:101F1000108275836483738362834183478346831E
:101F20000895CF93DF93DC019C91ED01898198178F
:101F300018F080E090E016C0ED01EC81FD81619326
:101F40008F81815019F48981E81BF109ED018F839C
:101F5000FD83EC839FB7F8948C918F5F8C939FBF28
:101F600081E090E0DF91CF910895FC01808188238A
:101F7000E9F3CF010E946B0F99270895FC0180813E
:101F8000882319F48FEF9FEF0895CF010E946B0F04
:101F90009927089581E090E0089581E090E0089508
:101FA00081E090E0089581E090E00895CF93DF9381
:101FB000CDB7DEB722970FB6F894DEBF0FBECDBF08
:101FC000982F8150833120F08751833108F07EC0F3
:101FD000E92FFF27EB5BFC4F82E08183892F992754
:101FE000AA27BB27FC013197EC32F10508F06EC03F
:101FF000EA5BFF4FEE0FFF1F0590F491E02D09946F
:10200000159A5BC0169A5DC0179A57C0B89A59C006
:10201000B99A53C0BA9A55C0BB9A4FC0BC9A51C026
:10202000BD9A4BC0BE9A4DC0BF9A47C0889A49C05E
:10203000899A43C08A9A45C08B9A3FC08C9A41C006
:102040008D9A3BC08E9A3DC08F9A37C0A09A39C0F6
:10205000A19A33C0A29A35C0A39A2FC0A49A31C0C6
:10206000A59A2BC0A69A2DC080916100806807C0F8
:1020700080916100806419C08091610080628093CA
:1020800061001BC08091610080610FC08091610080
:102090008860F5CF80916100846007C08091610005
:1020A0008260EDCF8091610081608093610009C002
:1020B000109A03C0119A05C0129A81E090E008C0FE
:1020C000139AE1E0F0E0FA83E98304C084E090E051
:1020D0009A83898389819A8122960FB6F894DEBF0C
:1020E0000FBECDBFDF91CF910895982F81508331DE
:1020F00030F08751833118F084E090E00895892F03
:102100000E94D60F81E090E00895CF93DF93CDB782
:10211000DEB722970FB6F894DEBF0FBECDBF982F63
:102120008150833120F08751833108F07EC0E92F40
:10213000FF27EB5BFC4F81E08183892F9927AA273A
:10214000BB27FC013197EC32F10508F06EC0EE5868
:10215000FF4FEE0FFF1F0590F491E02D09941598A5
:102160005BC016985DC0179857C0B89859C0B99809
:1021700053C0BA9855C0BB984FC0BC9851C0BD98C9
:102180004BC0BE984DC0BF9847C0889849C0899839
:1021900043C08A9845C08B983FC08C9841C08D98A9
:1021A0003BC08E983DC08F9837C0A09839C0A19889
:1021B00033C0A29835C0A3982FC0A49831C0A59869
:1021C0002BC0A6982DC0809161008F7707C08091A9
:1021D00061008F7B19C0809161008F7D80936100C9
:1021E0001BC0809161008F7E0FC080916100877F4E
:1021F000F5CF809161008B7F07C0809161008D7F5A
:10220000EDCF809161008E7F8093610009C01098AE
:1022100003C0119805C0129881E090E008C013989F
:10222000E1E0F0E0FA83E98304C084E090E09A837F
:10223000898389819A8122960FB6F894DEBF0FBEFA
:10224000CDBFDF91CF910895FB011082833091F0D3
:10225000843028F4813051F0823029F409C0843070
:1022600059F0853059F085E090E0089586B307C0B5
:1022700083B305C080B303C081B101C080B1808346
:1022800081E090E00895833091F0843028F481302B
:1022900051F0823029F409C0843059F0853069F05A
:1022A00084E090E0089568BB05C065BB03C062BBD5
:1022B00001C063B981E090E008956093620081E01D
:1022C00090E00895982FE82FFF27EB5BFC4F81816A
:1022D000823019F086E090E00895892F9927AA2787
:1022E000BB27FC013197EC32F10540F4E256FF4F79
:1022F000EE0FFF1F0590F491E02D099484E090E02B
:102300000895662311F01D9AFFC01D98FDC0662335
:1023100011F01E9AF9C01E98F7C0662311F01F9A9B
:10232000F3C01F98F1C0662311F0C09AEDC0C098A9
:10233000EBC0662311F0C19AE7C0C198E5C06623DF
:1023400011F0C29AE1C0C298DFC0662311F0C39AAF
:10235000DBC0C398D9C0662311F0C49AD5C0C49815
:10236000D3C0662311F0C59ACFC0C598CDC06623EF
:1023700011F0C69AC9C0C698C7C0662311F0C79AA3
:10238000C3C0C798C1C0662311F0909ABDC0909891
:10239000BBC0662311F0919AB7C09198B5C066236F
:1023A00011F0929AB1C09298AFC0662311F0939A3F
:1023B000ABC09398A9C0662311F0949AA5C09498D5
:1023C000A3C0662311F0959A9FC095989DC066237F
:1023D00011F0969A99C0969897C0662311F0979A33
:1023E00093C0979891C0662311F0A89A8DC0A898C1
:1023F0008BC0662311F0A99A87C0A99885C066236F
:1024000011F0AA9A81C0AA987FC0662311F0AB9AF6
:102410007BC0AB9879C0662311F0AC9A75C0AC98BC
:1024200073C0662311F0AD9A6FC0AD986DC066237E
:1024300011F0AE9A69C0AE9867C0662321F0809112
:10244000620080680DC0809162008F7709C06623AA
:1024500021F080916200806403C0809162008F7BD4
:102460008093620051C0662321F0809162008062F7
:10247000F7CF809162008F7DF3CF662321F08091AA
:1024800062008061EDCF809162008F7EE9CF66238C
:1024900021F0809162008860E3CF80916200877FA5
:1024A000DFCF662321F0809162008460D9CF8091D4
:1024B00062008B7FD5CF662321F08091620082601D
:1024C000CFCF809162008D7FCBCF662321F08091AA
:1024D00062008160C5CF809162008E7FC1CF66238C
:1024E00011F0189A11C018980FC0662311F0199AAC
:1024F0000BC0199809C0662311F01A9A05C01A98E2
:1025000003C0662321F01B9A81E090E008951B9898
:1025100081E090E008951F93182F8150833130F0AF
:102520008751833118F084E090E00FC0E12FFF273E
:10253000EB5BFC4F83E08183812F0E94D60F61E02B
:10254000812F0E94621181E090E01F910895CF9346
:10255000DF93982FEB011882E82FFF27EB5BFC4FEE
:102560008181813019F086E090E07DC0892F992724
:10257000AA27BB27FC013197EC32F10540F4E65362
:10258000FF4FEE0FFF1F0590F491E02D099484E0BA
:1025900090E069C00D9B65C062C00E9B62C05FC0C9
:1025A0000F9B5FC05CC0B09B5CC059C0B19B59C061
:1025B00056C0B29B56C053C0B39B53C050C0B49BCF
:1025C00050C04DC0B59B4DC04AC0B69B4AC047C025
:1025D000B79B47C044C0809B44C041C0819B41C061
:1025E0003EC0829B3EC03BC0839B3BC038C0849BA7
:1025F00038C035C0859B35C032C0869B32C02FC0E5
:10260000879B2FC02CC0989B2CC029C0999B29C0A8
:1026100026C09A9B26C023C09B9B23C020C09C9BA6
:1026200020C01DC0079B1DC01AC0069B1AC017C042
:10263000059B17C014C0049B14C011C0039B11C09C
:102640000EC0029B0EC00BC0089B0BC008C0099BAC
:1026500008C005C00A9B05C002C00B9B02C081E0F8
:10266000888381E090E0DF91CF910895CF93DF934D
:10267000CDB7DEB721970FB6F894DEBF0FBECDBF42
:102680009BE19093EB04BE016F5F7F4F0E94A71206
:102690008093EC0489818093ED041092EE0484E031
:1026A00090E00E94AE0121960FB6F894DEBF0FBEF7
:1026B000CDBFDF91CF9108959AE19093EB040E94F2
:1026C00062118093EC041092ED0483E090E00E948C
:1026D000AE01089598E19093EB040E94431180931A
:1026E000EC041092ED0483E090E00E94AE010895A6
:1026F000982F89E18093EB04933099F0943028F47B
:10270000913059F0923029F40AC0943061F095303C
:1027100061F085E090E020E00BC026B307C023B352
:1027200005C020B303C021B101C020B181E090E019
:102730008093EC042093ED041092EE0484E090E08A
:102740000E94AE01089597E19093EB040E948B12D2
:102750008093EC041092ED0483E090E00E94AE01BF
:10276000089595E19093EB040E9485108093EC040A
:102770001092ED0483E090E00E94AE01089596E18E
:102780009093EB040E94D60F8093EC041092ED041A
:1027900083E090E00E94AE01089584E18093EB0411
:1027A00081E08093EC041092ED0483E090E00E94BD
:1027B000AE01089582E18093EB0481E08093EC0404
:1027C0001092ED0483E090E00E94AE01089583E151
:1027D0008093EB0481E08093EC041092ED0483E09D
:1027E00090E00E94AE01089580E18093EB0481E0C7
:1027F0008093EC041092ED0483E090E00E94AE011F
:10280000089591E19093EB040E9475108093EC047D
:102810001092ED0483E090E00E94AE010895FC0167
:1028200080818531C9F1863180F4823131F1833183
:1028300030F48031D1F0813109F04CC01AC08331BD
:1028400009F1843109F046C022C0883189F189310B
:1028500028F4863129F18731E9F526C08A3189F1DA
:102860008A3158F18B31B1F531C082810E94F41365
:10287000089582810E9401140895638182810E94DB
:10288000DA130895638182810E94E71308956381BA
:1028900082810E94CD13089582810E94B113089510
:1028A00082810E94BF13089582810E94A31308951C
:1028B000638182810E946A13089582810E94781345
:1028C0000895638182810E945C13089582810E9431
:1028D000361308958093EB0483E08093EC04109208
:1028E000ED0483E090E00E94AE010895E82F81524C
:1028F000883018F084E090E00895FF27EB5BFC4FF0
:1029000084E0818381E090E00895E82FFF27EB5B6E
:10291000FC4F8181843019F084E090E008951182A9
:1029200081E090E0089517B8823039F0833049F0A3
:10293000813021F082E090E008953E9A81E090E0BD
:10294000089587B1806C87B981E090E0089593E89D
:1029500096B997B1907F982B97B9369A3699FECF52
:1029600084B195B120E030E040E050E0369A3699ED
:10297000FECF84B195B1480F591F2F5F3F4F2430D0
:102980003105A1F73798CA01969587959695879551
:102990000895CF93DF93EB0119821882282F3327F4
:1029A000F901EB5BFC4F8181843019F086E090E007
:1029B0000AC088E290E0821B930B0E94A7149983BF
:1029C000888381E090E0DF91CF91089593E2909326
:1029D000EB040E9493148093EC041092ED0483E0C6
:1029E00090E00E94AE010895CF93DF93CDB7DEB79C
:1029F00022970FB6F894DEBF0FBECDBF92E2909340
:102A0000EB04BE016F5F7F4F0E94C9148093EC04FA
:102A100029813A81832F99278093ED042093EE0436
:102A20001092EF0485E090E00E94AE0122960FB66E
:102A3000F894DEBF0FBECDBFDF91CF91089591E234
:102A40009093EB04E82FFF27EB5BFC4F81818430F0
:102A500019F084E090E003C0118281E090E080935F
:102A6000EC041092ED0483E090E00E94AE01089522
:102A7000E82F80E28093EB048E2F8152883018F08B
:102A800084E090E007C0FF27EB5BFC4F84E081838C
:102A900081E090E08093EC041092ED0483E090E0FC
:102AA0000E94AE010895FC018081813271F0823272
:102AB00018F48032B1F405C0823259F0833289F4BF
:102AC0000CC082810E943815089582810E941F15D2
:102AD000089582810E94F414089582810E94E61470
:102AE00008958093EB0483E08093EC041092ED044E
:102AF00083E090E00E94AE010895E4E7F0E0808179
:102B0000846080838BE0809352038CE08093530336
:102B100081E090E00895E4E7F0E080818B7F80839E
:102B2000109252031092530381E090E00895809335
:102B30007000E1E7F0E080818C7F8083808180837A
:102B400081E090E00895809171009927887F9070CE
:102B500008958091710084EA8093740080917400DC
:102B600087FFFCCF81E090E0089584E980937400B2
:102B70008091740084FDFCCF81E090E00895AC0169
:102B800020E030E00FC0FA01E20FF31F8081809354
:102B9000730084E8809374008091740087FFFCCFF9
:102BA0002F5F3F4F2617370774F3089584E880930B
:102BB00074008091740087FFFCCF80917300992787
:102BC000089585E38093EB0481E08093EC0420E09A
:102BD00030E00FC084E8809374008091740087FF18
:102BE000FCCF80917300F901E351FB4F80832F5F8D
:102BF0003F4F2617370774F3FB01E351FB4F108259
:102C0000CB0103960E94AE0108959B01BC01C9014E
:102C10000E94BF1581E08093EC041092ED0483E0E4
:102C200090E00E94AE01089584E980937400809141
:102C3000740084FDFCCF81E08093EC041092ED04DD
:102C400083E090E00E94AE0108958091710084EAD3
:102C5000809374008091740087FFFCCF81E08093A3
:102C6000EC041092ED0483E090E00E94AE01089520
:102C700080937000E1E7F0E080818C7F8083808129
:102C8000808381E08093EC041092ED0483E090E077
:102C90000E94AE010895E4E7F0E080818B7F80839D
:102CA000109252031092530381E08093EC0410922F
:102CB000ED0483E090E00E94AE010895E4E7F0E0C7
:102CC0008081846080838BE0809352038CE08093CA
:102CD000530381E08093EC041092ED0483E090E0D4
:102CE0000E94AE010895FC0180818093EB0484333F
:102CF000D1F0853338F4813379F0823381F0803339
:102D000031F507C08633E9F08633A0F08733F9F454
:102D10001BC00E945E1608950E944B160895828182
:102D20000E943816089582813396BF0199270E9428
:102D30000516089563817727828199270E94E115FE
:102D400008950E94251608950E941416089583E0A0
:102D50008093EC041092ED0483E090E00E94AE01B9
:102D60000895782F613079F0613050F0623021F0B1
:102D7000633009F059C002C061E003C061E004C0E3
:102D800060E030E002C060E031E04330D9F0443030
:102D900028F4413089F0423090F40CC0453031F0D5
:102DA0004530A0F0463009F03FC002C040E005C009
:102DB00040E006C041E007C041E050E005C041E00E
:102DC00050E006C040E051E020E003C040E051E0A8
:102DD00021E0BB9887B3866087BB88B3817F88BBBF
:102DE00080E090E0772311F081E090E075E0880FBB
:102DF000991F7A95E1F78065660F660F660F682B5D
:102E0000330F330F362B352B440F432B4DB92EB9CF
:102E100088E080934B038AE080934C0389E08093A1
:102E20004D0381E090E0089582E090E008951DB8A0
:102E30001EB810924B0310924C0310924D0381E088
:102E400090E00895AC0120E030E008C0E60FF71FE5
:102E500080818FB9779BFECF2F5F3F4FE22FFF27F7
:102E6000E417F5079CF381E090E00895DC0120E091
:102E700030E040E050E014C01FB809C083E0493E94
:102E800058071CF088E090E008954F5F5F4F779BF4
:102E9000F5CFFB01E20FF31F8FB180832F5F3F4F10
:102EA0002A173B074CF381E090E00895CF93DF931E
:102EB000EC0120E030E0A0E0B0E017C0FE01E20F3E
:102EC000F31F80818FB908C0119683E0A93EB8072F
:102ED0001CF088E090E00EC0779BF6CFFB01E20F7C
:102EE000F31F8FB180832F5F3F4F2417350734F3D3
:102EF00081E090E0DF91CF910895EF92FF920F93E0
:102F00001F938B01EBEEEE2EE4E0FE2E23E42093E4
:102F1000EB04B7016E5F7F4FA8010E9456178093A4
:102F2000EC040E5F1F4FE00EF11EF7011082C80186
:102F300001960E94AE011F910F91FF90EF900895AE
:102F4000EF92FF920F931F938C01FBEEEF2EF4E0B4
:102F5000FF2E84E48093EB04B7016E5F7F4FC801BE
:102F60000E9436178093EC040E5F1F4FE00EF11E97
:102F7000F7011082C80101960E94AE011F910F91C6
:102F8000FF90EF90089593E49093EB0499270E94AB
:102F900022178093EC041092ED0483E090E00E94ED
:102FA000AE01089581E48093EB040E94171780938B
:102FB000EC041092ED0483E090E00E94AE010895CD
:102FC00090E49093EB040E94B1168093EC0410926D
:102FD000ED0483E090E00E94AE010895CF93DF936B
:102FE000EC0188818334A9F0843428F4803441F0E2
:102FF000813409F50BC0843499F08534E1F414C0B0
:103000004C816B818A810E94E01720C00E94D217F8
:103010001DC0BE016D5F7F4F8A810E94C31716C01D
:103020008A8199270E94A0176A817727CE0103968B
:103030000E947D170BC08093EB0483E08093EC0427
:103040001092ED0483E090E00E94AE01DF91CF91F9
:103050000895B89AB99ABA9ABB98BC9ABD9AC4987E
:10306000C59881E08093560382E080935703809354
:1030700058038093590381E090E00895109256031D
:1030800010925703109258031092590381E090E078
:103090000895C098C198C29880E29EE40197F1F724
:1030A000C09A8AE0982F9A95F1F7C29AC19A8A95A8
:1030B000F1F70895282FC19887FD02C0C29801C07A
:1030C000C29A8AE0982F9A95F1F7C19A8A95F1F7FA
:1030D000C19826FF02C0C29A01C0C2988AE0982F08
:1030E0009A95F1F7C19A8A95F1F70895282F220F42
:1030F00030E0C19827FF02C0C29A01C0C2988AE09E
:10310000982F9A95F1F7C19A8A95F1F73F5F37307A
:1031100011F0220FEECF0895282F30E0C19827FF3D
:1031200002C0C29A01C0C2988AE0982F9A95F1F71E
:10313000C19A8A95F1F73F5F383011F0220FEECF38
:103140000895C198C2988AE0982F9A95F1F7C19A8C
:10315000982F9A95F1F7C198C098982F9A95F1F702
:10316000C19A982F9A95F1F7C1988A95F1F7C09A6C
:1031700080E090E00895C198C098C298C39A0895DD
:103180000E94491880E30E945A1880E60E9476182F
:1031900008950E94491880E00E945A1880E00E9419
:1031A00076180E94BB1808950F931F93182F062FAF
:1031B0000E94491880E40E945A18812F0E947618B4
:1031C000802F0E948C1881E090E01F910F9108954C
:1031D0001F93182F0E94491880EC0E945A18812FC3
:1031E0000E9476180E94A11899271F910895C198EE
:1031F0008AE08A95F1F7C29830E090E0990FC19A81
:103200002AE0822F8A95F1F7C198B3999F5F822FA8
:103210008A95F1F73F5F383089F7C098C19A822FBD
:103220008A95F1F7C09AC1982A95F1F7892F9927C5
:1032300008951F93182F0E94491880E80E945A1879
:10324000812F0E9476180E94F71899271F910895E0
:10325000DF92EF92FF920F931F93CF93DF93D82EBD
:103260007B018A01C0E0D0E009C08D2D8C0F0E9447
:103270001919F801EC0FFD1F80832196CE15DF058B
:10328000A1F781E090E0DF91CF911F910F91FF9026
:10329000EF90DF9008950F931F93082F162F0E9431
:1032A000C018612F802F0E94D41881E090E01F91F8
:1032B0000F910895DF92EF92FF920F931F93CF9398
:1032C000DF93D82E7B018A01C0E0D0E009C0F8016D
:1032D000EC0FFD1F60818D2D8C0F0E944B192196E4
:1032E000CE15DF05A1F781E090E0DF91CF911F912E
:1032F0000F91FF90EF90DF90089594E09093EB048E
:103300000E945A198093EC041092ED0483E090E03F
:103310000E94AE010895EF92FF920F931F938B01CD
:103320009BEEE92E94E0F92E93E09093EB04A70135
:103330004E5F5F4F0E9428198093EC040E5F1F4F71
:10334000E00EF11EF7011082C80101960E94AE0145
:103350001F910F91FF90EF90089582E08093EB040E
:10336000109256031092570310925803109259036B
:1033700081E08093EC041092ED0483E090E00E94E1
:10338000AE01089581E08093EB040E942918809398
:10339000EC041092ED0483E090E00E94AE010895E9
:1033A000FC018381823069F0833018F48130F1F4BC
:1033B00005C0833049F08430C9F40FC00E94C2199F
:1033C00008950E94AD190895AF014A5F5F4F65816E
:1033D000772784810E948B190895AF014A5F5F4F60
:1033E0006581772784810E947D190895808180936B
:1033F000EB0483E08093EC041092ED0483E090E012
:103400000E94AE0108951F920F920FB60F921124E1
:103410000F900FBE0F901F9018959C010897029770
:1034200018F084E090E00895F901EB5BFC4F8DE02B
:1034300081832830310561F02930310519F087E0AA
:1034400090E00895BD9A81E090E09BBD8ABD08950B
:10345000BC9A81E090E00895FC01EB5BFC4F118287
:1034600081E090E008959C01FC01EB5BFC4F8181C1
:103470008D3019F086E090E008952830310539F15B
:103480002930310519F087E090E008956330710527
:10349000A9F0643071053CF46130710559F0623077
:1034A0007105A9F409C06430710551F065307105EA
:1034B00071F408C081E007C082E005C083E003C06A
:1034C00084E001C085E08EBD81E090E0089581E058
:1034D00090E008959C01FC01EB5BFC4F81818D30F5
:1034E00019F086E090E008952830310531F0293058
:1034F000310531F087E090E0089581E090E0089593
:103500007BBD6ABD81E090E008959C0183E58093D6
:10351000EB04F901EB5BFC4F81818D3019F086E003
:1035200090E00DC02830310541F02930310519F007
:1035300087E090E004C07BBD6ABD81E090E08093AD
:10354000EC041092ED0483E090E00E94AE01089537
:1035500022E52093EB040E94331A8093EC0410922E
:10356000ED0483E090E00E94AE01089521E52093F0
:10357000EB04FC01EB5BFC4F118281E08093EC04D7
:103580001092ED0483E090E00E94AE01089520E5E2
:103590002093EB040E940D1A8093EC041092ED042A
:1035A00083E090E00E94AE010895FC0180818135A6
:1035B00079F0823518F48035F1F405C0823569F070
:1035C0008335C9F411C0828199270E94C71A0895D2
:1035D000828199270E94B61A089563817727828194
:1035E00099270E94A81A08956381772782819927D5
:1035F0000E94851A08958093EB0483E08093EC0485
:103600001092ED0483E090E00E94AE010895CF9304
:10361000DF93CDB7DEB7DF91CF910895089581E0B4
:1036200090E0089508958A3310F4805301C08755BF
:103630006A3310F4605301C067556F708295807FC4
:10364000682B862F992708950895DC0180E1A0302A
:10365000B80718F082E090E00895E199FECF9D014F
:1036600009C03FBB2EBB2F5F3F4FE09AE60FF71F0D
:103670008DB38083822F8A1BE82FFF27E417F5077D
:1036800080F381E090E00895DC0180E1A030B8078C
:1036900018F082E090E00895E199FECF9D010AC004
:1036A0003FBB2EBB2F5F3F4FE60FF71F80818DBBC7
:1036B000E29AE19A822F8A1BE82FFF27E417F50789
:1036C00078F381E090E008950F931F938B0121E838
:1036D0002093EB040E94441B8093EC041092ED04B1
:1036E0001F930F9389EF92E09F938F930E94071B84
:1036F00083E090E00E94AE010F900F900F900F902A
:103700001F910F910895CF92DF92EF92FF920F9346
:103710001F937B010BEE14E020E82093EB0422E0E2
:10372000C22ED12CC00ED11EAB01B6010E94251BAA
:103730008093EC0482E090E0E80EF91E0E0D1F1D50
:10374000F8011082DF92CF9286E093E09F938F93EF
:103750000E94071BC70101960E94AE010F900F90B7
:103760000F900F901F910F91FF90EF90DF90CF90EF
:103770000895EF92FF920F931F93CF93DF93EC0185
:103780008B819927F82EEE248A81E80EF11C8D8119
:103790009927182F00278C81080F111DFF92EF9297
:1037A0001F930F9380E193E09F938F930E94071BD9
:1037B00088812DB73EB72A5F3F4F0FB6F8943EBFC2
:1037C0000FBE2DBF803819F0813869F405C0B801EB
:1037D000C7010E94831B12C02696A801BE01C70123
:1037E0000E94641B0BC08093EB0483E08093EC0485
:1037F0001092ED0483E090E00E94AE01DF91CF9142
:103800001F910F91FF90EF900895CF93DF93AC013C
:10381000029710F442E050E0A0917006B09171065A
:10382000FD01C0E0D0E020E030E020C08081918147
:103830008417950769F482819381209719F09B83FF
:103840008A8304C090937106809370069F0132C0F2
:103850004817590738F42115310519F082179307D5
:1038600008F49C01EF010280F381E02D3097F1F61E
:103870002115310599F1C901841B950B049708F4B2
:10388000A901E0E0F0E028C08D919C91119782178A
:103890009307F9F44817590781F4ED018A819B8158
:1038A000309719F09383828304C0909371068093BC
:1038B00070069D012E5F3F4F4CC0841B950BFD0190
:1038C000E80FF91F4193519302978D939C939F01A9
:1038D00040C0FD01A281B3811097B1F680916E06C0
:1038E00090916F06892B41F48091370390913803B2
:1038F00090936F0680936E062091390330913A03BE
:103900002115310549F48DB7282F332780913503D0
:1039100090913603281B390BA0916E06B0916F066B
:103920002A1B3B0B2417350790F0CA010296281773
:10393000390768F09D012E5F3F4FC901840F951F25
:1039400090936F0680936E064D935C9302C020E0C7
:1039500030E0C901DF91CF910895CF93DF930097B5
:1039600009F44EC0EC0122971B821A82A0917006C6
:10397000B0917106109711F140E050E001C0DC01F8
:10398000AC17BD0700F1BB83AA83FE0121913191E1
:10399000E20FF31FEA17FB0771F48D919C911197C9
:1039A000280F391F2E5F3F4F39832883FD01828105
:1039B00093819B838A834115510559F4D0937106F5
:1039C000C09370061DC0FD0182819381AD010097F7
:1039D000B1F6FA01D383C28321913191E20FF31F33
:1039E000EC17FD0769F488819981280F391F2E5F34
:1039F0003F4FFA01318320838A819B8193838283A5
:103A0000DF91CF91089597FB092E07260AD077FD05
:103A100004D00CD006D000201AF4709561957F4F29
:103A20000895F6F7909581959F4F0895AA1BBB1BAB
:103A300051E107C0AA1FBB1FA617B70710F0A61BAE
:103A4000B70B881F991F5A95A9F780959095BC01CF
:063A5000CD010895FFCF37
:103A5600456D62656464656450726F6A656374730C
:103A6600004F63746F70757355534220496E7465C9
:103A7600726661636520436F6E7665727465722047
:103A8600616E6420492F4F20457874656E73696FA7
:103A96006E003230303831313038006669727374F6
:103AA600207061636B6574206F662061206C6F6E99
:103AB60067206D65737361676520286C656E677432
:103AC600683A202564290A006F63746F7075732045
:103AD6006C6F6E672072756E6E696E67206D6573AA
:103AE600736167650A006F63746F7075732E6C6F10
:103AF6006E675F696E646578203C206F63746F70D3
:103B060075732E6C6F6E675F62797465730A006EEB
:103B16006F74206C617374207061636B65743A20F6
:103B260064696666203E2036340A006C6173742030
:103B36007061636B65740A007061727365722C2024
:103B4600636865636B3A2025582C20636F6D6D6141
:103B56006E643A2025580A0063616C6C696E6720B2
:103B6600696F5F7061727365720A0063616C6C697C
:103B76006E67206164635F7061727365720A0063C9
:103B8600616C6C696E67206932635F706172736520
:103B9600720A0063616C6C696E67207370695F708E
:103BA60061727365720A0063616C6C696E6720707E
:103BB600776D5F7061727365720A0063616E277458
:103BC6002063616C6C2063616E5F706172736572F5
:103BD600202D206E6F2043414E2D737570706F72CD
:103BE600740A0063616C6C696E6720656570726F3C
:103BF6006D5F7061727365720A00756E6B6E6F77BA
:103C06006E20636D640A00726563656976696E6726
:103C160020636F6D6D616E643A20255820286C65AF
:103C26006E6774683A202575290A00676574206EE8
:103C36006578740A0067657420616E64206578652E
:103C4600637574650A000904007772697474656E99
:103C56003A2025730A00726561643A2025730A00CA
:103C6600656570726F6D5F7061727365723A206C14
:103C7600656E6774683A2025752C20616464723A13
:0C3C86002025750A0020007206000000D6
:00000001FF
